:100000000C945B000C9402020C942F020C9483005D
:100010000C9483000C9483000C9483000C94830054
:100020000C9483000C9483000C9483000C94830044
:100030000C9483000C9483000C9483000C94830034
:100040000C945C020C9483000C9445040C94830083
:100050000C9483000C9483000C9483000C94830014
:100060000C9483000C948300000024272A000025B0
:10007000282B000023262904040404040404040299
:100080000202020202030303030303010204081035
:100090002040800102040810200102040810200002
:1000A0000000070002010000030406000000000039
:1000B00000000000F70111241FBECFEFD4E0DEBF27
:1000C000CDBF11E0A0E0B1E0E2E6F9E002C00590AA
:1000D0000D92A631B107D9F711E0A6E1B1E001C058
:1000E0001D92AC3AB107E1F710E0C6EBD0E004C0D6
:1000F0002297FE010E94AB04C43BD107C9F70E94BE
:10010000F0010C94AF040C940000EF92FF920F9357
:100110001F93CF93DF93809100010E94F1037C0134
:10012000809102010E94F1038C01809104010E94E0
:10013000F103EC01809106010E94F10320E030E020
:10014000892B11F421E030E0220F331F80E090E092
:10015000CD2B11F481E090E0280F391F220F331FBF
:1001600080E090E0012B11F481E090E0280F391F2E
:10017000220F331F80E090E0EF2811F481E090E03F
:10018000280F391FC901DF91CF911F910F91FF9067
:10019000EF90089560E070E080910C010E943003C0
:1001A00060E070E080910A010E94300360E070E03E
:1001B00080910E010E943003089560E070E080910C
:1001C0000C010E9430036FEF70E080910A010E94E1
:1001D000300360E070E080910E010E9430030895CA
:1001E00060E070E080910C010E94300362E370E0F7
:1001F00080910A010E9430036FEF70E080910E0140
:100200000E943003089567EF70E080910C010E9416
:1002100030036CE170E080910A010E94300366EBCC
:1002200070E080910E010E94300308956FEF70E03E
:1002300080910C010E94300360E070E080910A011F
:100240000E94300360E070E080910E010E94300354
:1002500008956FEF70E080910C010E9430036FEF02
:1002600070E080910A010E94300360E070E08091AC
:100270000E010E94300308956FEF70E080910C0131
:100280000E9430036FEF70E080910A010E943003FA
:100290006FEF70E080910E010E94300308950E947C
:1002A0008500009719F40E94CA00089581309105D5
:1002B00019F40E94290108958230910519F40E94D1
:1002C000160108958330910519F40E9403010895E1
:1002D0008430910519F40E94F0000895853091054D
:1002E00019F40E94DD0008950F9711F40E943C015B
:1002F00008950E944F016AE070E080E090E00E9463
:10030000CC02089561E0809108010E94A60364E692
:1003100070E080E090E00E94CC0260E080910801F3
:100320000E94A603089560E0809100010E94880366
:1003300060E0809102010E94880360E080910401E6
:100340000E94880360E0809106010E94880361E0BA
:10035000809108010E94880361E080910C010E9455
:10036000880361E080910A010E94880361E0809126
:100370000E010E9488030E943C0168EE73E080E059
:1003800090E00E94CC020E94290168EE73E080E0B8
:1003900090E00E94CC020E94160168EE73E080E0BB
:1003A00090E00E94CC020E94030168EE73E080E0BE
:1003B00090E00E94CC020E94F00068EE73E080E0C2
:1003C00090E00E94CC020E94DD0068EE73E080E0C5
:1003D00090E00E94CC020E94CA000E94820108950F
:1003E0000E94F6020E9493010E947901FDCF84E1F0
:1003F00091E090931701809316010895862F0E9433
:100400003D0408951F920F920FB60F9211242F935F
:100410003F934F935F936F937F938F939F93AF938C
:10042000BF93EF93FF938091180190911901892B4D
:1004300029F0E0911801F09119010995FF91EF91D0
:10044000BF91AF919F918F917F916F915F914F91EC
:100450003F912F910F900FBE0F901F9018951F92F4
:100460000F920FB60F9211242F933F934F935F93E8
:100470006F937F938F939F93AF93BF93EF93FF936C
:1004800080911A0190911B01892B29F0E0911A01AA
:10049000F0911B010995FF91EF91BF91AF919F9151
:1004A0008F917F916F915F914F913F912F910F901D
:1004B0000FBE0F901F9018951F920F920FB60F92BC
:1004C00011242F938F939F93AF93BF9380911C011F
:1004D00090911D01A0911E01B0911F010196A11DD7
:1004E000B11D80931C0190931D01A0931E01B09338
:1004F0001F018091200190912101A0912201B091D2
:1005000023018050904CAF4FBF4F809320019093B8
:100510002101A0932201B093230127C080912001E3
:1005200090912101A0912201B091230180589E4316
:10053000A040B0408093200190932101A09322011C
:10054000B09323018091240190912501A09126016F
:10055000B09127010196A11DB11D809324019093B4
:100560002501A0932601B09327018091200190914D
:100570002101A0912201B091230181589E43A04006
:10058000B04060F6BF91AF919F918F912F910F90E6
:100590000FBE0F901F901895EF92FF920F931F932D
:1005A0007B018C018FB7F894409124015091250173
:1005B00060912601709127018FBF2FB7F894809129
:1005C000240190912501A0912601B09127012FBF10
:1005D000841B950BA60BB70BE816F9060A071B0739
:1005E00060F71F910F91FF90EF900895789484B574
:1005F000826084BD84B5816084BD85B5826085BD1F
:1006000085B5816085BDEEE6F0E080818160808304
:10061000E1E8F0E080818260808380818160808376
:10062000E0E8F0E0808181608083E1EBF0E08081B0
:1006300084608083E0EBF0E0808181608083EAE782
:10064000F0E080818460808380818260808380810B
:10065000816080838081806880831092C1000895CA
:100660001F93CF93DF93182FEB0161E00E94880363
:10067000E12FF0E0E156FF4F8491833051F48091F7
:100680008000806880938000D0938900C0938800A8
:100690003BC0843051F48091800080628093800060
:1006A000D0938B00C0938A002FC0813039F42097FB
:1006B00029F184B5806884BDC7BD26C0823039F475
:1006C0002097E1F084B5806284BDC8BD1DC086302E
:1006D00041F48091B00080688093B000C093B30073
:1006E00013C0873041F48091B00080628093B000E5
:1006F000C093B40009C0C038D10514F460E001C053
:1007000061E0812F0E94A603DF91CF911F91089590
:10071000282F30E0C90185579F4FFC01949129583B
:100720003F4FF9018491882381F0E82FF0E0E859E8
:10073000FF4FE491F0E0662329F4808190958923AE
:10074000808308958081892B80830895482F50E00D
:10075000CA0181569F4FFC012491CA0185579F4FC2
:10076000FC01949149585F4FFA0134913323C1F150
:10077000222331F1233021F4809180008F7705C04E
:10078000243031F4809180008F7D8093800018C0E8
:10079000213019F484B58F7704C0223021F484B558
:1007A0008F7D84BD0DC0263021F48091B0008F77FD
:1007B00005C0273029F48091B0008F7D8093B00070
:1007C000E32FF0E0E359FF4FE491F0E0662329F4D2
:1007D000808190958923808308958081892B8083EF
:1007E0000895482F50E0CA0181569F4FFC01249183
:1007F000CA0185579F4FFC01949149585F4FFA01F8
:100800003491332319F420E030E035C0222331F154
:10081000233021F4809180008F7705C0243031F49B
:10082000809180008F7D8093800018C0213019F462
:1008300084B58F7704C0223021F484B58F7D84BDC8
:100840000DC0263021F48091B0008F7705C027308D
:1008500029F48091B0008F7D8093B000E32FF0E009
:10086000EE58FF4FE491F0E0808120E030E08923F2
:1008700011F021E030E0C9010895982F8091C00067
:1008800085FFFCCF9093C60008951F920F920FB67C
:100890000F9211242F933F934F935F936F937F9306
:1008A0008F939F93AF93BF93EF93FF934091C600B5
:1008B000E0912801F0912901CF01019660E870E0F4
:1008C0000E9482049C0180912A0190912B0128179B
:1008D000390739F0E45DFE4F4083309329012093BE
:1008E0002801FF91EF91BF91AF919F918F917F91DF
:1008F0006F915F914F913F912F910F900FBE0F908D
:100900001F90189597FB092E07260AD077FD04D073
:100910000CD006D000201AF4709561957F4F089591
:10092000F6F7909581959F4F0895AA1BBB1B51E147
:1009300007C0AA1FBB1FA617B70710F0A61BB70B4F
:10094000881F991F5A95A9F780959095BC01CD01F4
:100950000895EE0FFF1F0590F491E02D0994F8948F
:02096000FFCFC7
:100962000200030004000500060009000A000B0053
:0609720000000000FE0180
:00000001FF
